S00F000070776D746573312E7372656344
S11300000C942A000C9445000C9445000C94450073
S11300100C9445000C9445000C9445000C94450048
S11300200C9445000C9445000C9445000C94450038
S11300300C9445000C9445000C9445000C94450028
S11300400C9445000C9445000C9445000C94450018
S11300500C94450011241FBECFE5D8E0DEBFCDBF10
S113006010E0A0E6B0E0E8EBF1E002C005900D92EC
S1130070A037B107D9F710E0A0E7B0E001C01D92A6
S1130080A037B107E1F70C948A000C94000087E8CC
S113009086B90895877087B9369A3699FECF84B1A8
S11300A095B108950F931F93CF93DF9380E00E943F
S11300B04A0097FD22C0EC01D595C795D595C79503
S11300C081E00E944A0097FD23C08C011595079595
S11300D01595079580E690E00E94C6008C2F0E943B
S11300E0B10083E690E00E94C600802F0E94B10018
S11300F080E00E944A0097FFDECF0396EC01D5957D
S1130100C795D595C79581E00E944A0097FFDDCF3A
S11301100396DBCFCFE5D8E0DEBFCDBF17BA11BA67
S11301200E9447008FEC90E00E949E0086E690E0DB
S11301300E94C6000E9452000C94DB009C01832F95
S1130140992780BD29B988E18AB98EE880BD0895D0
S11301505F9BFECF8CB1992708955D9BFECF8CB930
S11301600895CF93982F82958F70805D8A3308F01D
S1130170895F9F70C92FC05DCA3308F0C95F0E94B0
S1130180AD008C2F0E94AD00CF910895CF93DF93E3
S1130190EC018881882361F089910E94AD008881F7
S11301A0882331F089910E94AD0088818823A1F7CA
S10B01B0DF91CF910895FFCF08
S11301B850580050590052454144592E0A0D000028
S9030000FC
